:100000000C944D010C946A010C946A010C946A01E1
:100010000C9473080C947F070C9446080C94EC071E
:100020000C9419080C9452070C94BF070C94FF060B
:100030000C946A010C9405030C946A010C94CE0292
:100040000C94EC080C946A010C946A010C946A01FB
:100050000C946A0130313233343536373839414205
:100060004344454600000001000800200040008095
:100070000000010004000001000800400000010031
:10008000041B63001B5B324A001B5B25646D001B75
:100090005B3F323568001B5B3F32356C001B5B25D4
:1000A000643B25644800636F6D6D616E64206E6F04
:1000B0007420666F756E6400636D646C696E653A7A
:1000C0002000633E0079A780E3888D90AB9946A21B
:1000D00063AC0BB646C11CCC98D8C3E5A680858B13
:1000E00091989EA5ADB5BDC5CEE7E0EAF580008646
:1000F000478C8B92C798F89F19A527AB1EB0FBB60B
:10010000B9BC56C1CDC71CCC3FD133D5F4DA81DEA2
:10011000D6E2F1E6CEEA6CEDC9F0E1F3B5F640F8CF
:1001200083FA7CFC29FD89FE9CFF61FFD7FFFEFF5F
:10013000D7FF61FE9CFD89FC29FA7CF883F640F329
:10014000B5F0E1EDC9EA6CE6CEE2F1DED6DA81D5B2
:10015000F5D133CC3FC71CC1CDBC56B6B9B0FBAB53
:100160001EA5279F1998F892C78C8B864780007927
:10017000B873746D38670760E65AD854E14F044984
:100180004643A93E3238E333C02ECC2A0B257E21CC
:10019000291D0E1931159312360F1E0C4B09BF077E
:1001A0007C058303D702760163009E0028000100CE
:1001B00028009E0163027603D60583077C09BF0CE5
:1001C0004A0F1E1236159319311D0E2129257E2A3C
:1001D0000A2ECC33C038E33E3243A949464F04547B
:1001E000E05AD860E667076D37737479B845656C77
:1001F00020636F6D6D616E647A210D0A0045786928
:100200007465642070726F6772616D210D0A00253C
:1002100064202020256420002564202020256420DF
:100220000D0A00696E702076616C203D2025640DFA
:100230000A00696E702076616C203D2025642020C4
:100240000D0A00256420006C6F776573744B657927
:100250003A20256420000D0A0025640D0A0025645B
:100260000D0A000D0A000D0A0028256429202564C6
:1002700020202020000D0A000D0A57656C636F6D69
:100280006520746F204372616E6B7363616C6521CE
:100290000D0A00256420000D0A0011241FBECFE5C1
:1002A000D8E0DEBFCDBF11E0A0E6B0E0EEE1FAE2BB
:1002B00002C005900D92A437B107D9F717E0A4E763
:1002C000B1E001C01D92AC37B107E1F70E946D119A
:1002D0000C940E150C940000FC019A014FB7F89491
:1002E000718360833383228317821682158214827E
:1002F0004FBF0895CF93DF93DC01E0E06FB7F89430
:10030000EC014C815D8141155105C9F0ED91FC91E5
:1003100011978E819F81E80FF91FE08101969F83DD
:100320008E832A813B818217930720F0821B930BD7
:100330009F838E8341505040ED015D834C836FBF9E
:100340008E2F9927DF91CF910895FC01AFB7F894D4
:100350004481558164177507A0F486819781860FC3
:10036000971F97838683228133818217930720F01A
:10037000821B930B97838683461B570B55834483BD
:1003800002C015821482AFBF08951F93FC011FB7EE
:10039000F8948681978122813381860F971FB90156
:1003A0000E947B140190F081E02DE80FF91F8081FD
:1003B0001FBF99271F9108951F93CF93DF93EC01DF
:1003C000162F4FB7F8942C813D816A817B812617C7
:1003D0003707A0F48E819F81820F931F0E947B14A8
:1003E000E881F981E80FF91F10838C819D810196C6
:1003F0009D838C834FBF8FEF90E003C04FBF80E0A1
:1004000090E0DF91CF911F910895FC014FB7F894D0
:1004100022813381848195814FBF281B390BC9010B
:100420000895FC018FB7F894158214828FBF089548
:10043000DC01CB0173E0880F991FAA1FBB1F7A95BF
:10044000D1F79C01AD01220F331F441F551F80506F
:100450009C4DAB40BF4FBC01CD010E948F14DA010F
:10046000C901019789B9892F992780BD089540E472
:1004700050E064E771E085EF94E00E946C0140E495
:1004800050E064EB71E08EEF94E00E946C010895FF
:100490000E9437021092F5011092F40188ED8AB99A
:1004A00060E875E280E090E00E9418028FEF809390
:1004B000F4041092FD04109207051092060578943A
:1004C00008959093F5018093F401089585EF94E0E9
:1004D00008958EEF94E00895982F8091F404882376
:1004E000E1F39CB91092F4040895CF93DF93EC01EB
:1004F0008091F7049091F804009769F08091F904D5
:100500009091FA04009739F085EF94E00E947A0107
:1005100088838FEF90E0DF91CF910895CF93DF93A1
:10052000CDB7DEB721970FB6F894DEBF0FBECDBFB3
:10053000CE0101960E947502882319F089819927BE
:1005400002C08FEF9FEF21960FB6F894DEBF0FBE6B
:10055000CDBFDF91CF9108951092FA041092F90463
:1005600008958091F9049091FA04892B19F48FEF82
:1005700090E0089580E090E00895682F8EEF94E079
:100580000E94DC01992708958FEF8093FD048EEF80
:1005900094E00E947A010E946C0208951F920F92CB
:1005A0000FB60F9211242F933F934F935F936F9346
:1005B0007F938F939F93AF93BF93EF93FF9380911C
:1005C000FD04882371F08091020590910305892B29
:1005D00031F08EEF94E00E947A018CB905C0109240
:1005E000FD048FEF8093F404FF91EF91BF91AF91E1
:1005F0009F918F917F916F915F914F913F912F913B
:100600000F900FBE0F901F9018951F920F920FB66C
:100610000F9211242F933F934F935F936F937F9388
:100620008F939F93AF93BF93EF93FF936CB18091A0
:10063000F4019091F501892B39F0E091F401F091EA
:10064000F501862F09950FC085EF94E00E94DC012B
:10065000882349F4809106059091070501969093AF
:10066000070580930605FF91EF91BF91AF919F9190
:100670008F917F916F915F914F913F912F910F904B
:100680000FBE0F901F9018959093F7018093F6017D
:100690000895CF93C82F8A3031F4E091F601F0919C
:1006A000F7018DE00995E091F601F091F7018C2FAB
:1006B0000995CF910895CF93DF93EC01892B49F0F1
:1006C0008881882331F089910E9449038881882399
:1006D000D1F7DF91CF910895EF92FF920F931F937F
:1006E000CF93DF938C017A01C0E0D0E0892BE9F051
:1006F000CE0121968617970728F4F80181918F0182
:100700008823B1F7C0E0D0E0CE15DF0570F4F80122
:100710008081882319F00F5F1F4F01C080E20E9483
:1007200049032196CE15DF0590F3DF91CF911F91FC
:100730000F91FF90EF900895CF93DF93EC01009716
:1007400061F0FC0121968491882339F00E944903CD
:10075000FE01219684918823C9F7DF91CF910895F6
:100760008AE00E9449030895E82FFF27EF70F07098
:10077000EC5AFF4F84910E94490308951F93182F4C
:1007800082958F700E94B403812F0E94B4031F9141
:1007900008950F931F938C01812F99270E94BE0308
:1007A000802F0E94BE031F910F910895EF92FF9238
:1007B0000F931F937B018C01C801AA27BB270E94BE
:1007C000C903C7010E94C9031F910F91FF90EF90C9
:1007D00008952F923F924F925F926F927F928F92E5
:1007E0009F92AF92BF92CF92DF92EF92FF920F93C0
:1007F0001F93CF93DF93CDB7DEB7A2970FB6F894D0
:10080000DEBF0FBECDBF69A3242E2AA33701480146
:10081000442351F017FF08C0EE24FF248701E61897
:10082000F7080809190902C08401730199A1692F09
:10083000772767FD709561507040222011F061505C
:100840007040362E18A22FE1422E512C4C0E5D1E08
:10085000A82EBB24A7FCB094CB2CDB2CC801B7017D
:10086000A60195010E948F14DC01CB01FC01EF7001
:10087000F070EC5AFF4F84918F8FC801B701A60129
:1008800095010E948F1479018A013A94EFEF3E1688
:1008900049F1C2010197E114F10401051105D1F0FC
:1008A0002C01C801B701A60195010E948F14DC013B
:1008B000CB01FC01EF70F070EC5AFF4F8491F20114
:1008C0008083C801B701A60195010E948F147901A8
:1008D0008A0104C02C018AA1F20180833A949FEF1F
:1008E0003916B9F62220A9F097FE05C08DE2F20173
:1008F00082932F010EC0C201019716141704180429
:1009000019041CF42C018BE202C02C0180E2F201DC
:10091000808339A03A94FFEF3F1649F0F2018191AC
:100920002F010E9449033A94FFEF3F16B9F7A296B0
:100930000FB6F894DEBF0FBECDBFDF91CF911F91F0
:100940000F91FF90EF90DF90CF90BF90AF909F906E
:100950008F907F906F905F904F903F902F90089571
:100960007F928F929F92AF92BF92CF92DF92EF923F
:10097000FF920F931F93CF93DF93CDB7DEB77888A5
:10098000C988DA8873E1A72EB12CAC0EBD1E05C054
:10099000882309F477C00E94490396012F5F3F4FD7
:1009A000772021F0F6016901849103C0F60180816E
:1009B0006901853269F72F5F3F4F772021F0F601FB
:1009C0006901849103C0F60180816901282F3327D2
:1009D00027FD30952436310591F02536310524F474
:1009E0002336310529F0D7CF2837310581F0D3CF11
:1009F000F50122E030E0A20EB31E8081CCCF6AE088
:100A0000862E912C50E1E52E57E2F52E06C040E1EE
:100A1000842E912CE12C30E1F32EF50122E030E020
:100A2000A20EB31E008111818436C1F417FF06C0E7
:100A3000109501951F4F8DE20E94490332E0E316A5
:100A4000F10460F00E151F0548F4C7016AE070E07C
:100A50000E947B147B0162307105A0F7C801B701C9
:100A60000E947B14CB010E94B403C801B7010E940D
:100A70007B148C01C701B4010E947B147B01672B9E
:100A800069F78BCF80E090E0DF91CF911F910F91BC
:100A9000FF90EF90DF90CF90BF90AF909F908F909E
:100AA0007F900895039665E070E00E947B14CB016F
:100AB000AA27BB2724E0880F991FAA1FBB1F2A95CE
:100AC000D1F720E030E02817390718F42F5F3F4FA7
:100AD000FACF0895883040F4E82FFF27EE0FFF1F6C
:100AE000E850FE4F11821082089593B7987F982B9B
:100AF00093BF0895109208051092090510920A05F7
:100B000010920B05089582E00E94750512BE89B708
:100B1000816089BF0E947A0508959EB5987F982BC1
:100B20009EBD089583E00E948D051DBC1CBC89B745
:100B3000846089BF089595B5987F982B95BD0895D9
:100B400010921005109211051092120510921305C3
:100B5000089584E00E949B0514BC89B7806489BF16
:100B60000E94A0050895CF93C0E08C2F0E946A05D3
:100B7000CF5FC830D0F30E9483050E9492050E9487
:100B8000A9057894CF91089583B7E82FFF27E770E0
:100B9000F070EE0FFF1FEB58FF4F85919491089571
:100BA0008EB5E82FFF27E770F070EE0FFF1FEB58B0
:100BB000FF4F85919491089585B5E82FFF27E77041
:100BC000F070EE0FFF1FEB59FF4F85919491089540
:100BD000883040F4E82FFF27EE0FFF1FE850FE4F4C
:100BE000718360830895DF92EF92FF920F931F93BA
:100BF000CF93DF93EC01D2B610920C0510920D0545
:100C000010920E0510920F050E94C4059C01442706
:100C1000552760E074E284EF90E00E94B114293B14
:100C20008DE8380786E0480780E05807C0F487E27F
:100C3000C131D807A0F4CE01AA27BB27BC01CD0142
:100C40000E945C14DC01CB01BC01CD0128EE33E035
:100C500040E050E00E948F14FA01E90111C07E01CA
:100C600000271127CA01B90128EE33E040E050E027
:100C70000E948F14C801B7010E945C14FC01EB01B3
:100C800080910C0590910D05A0910E05B0910F0576
:100C90002227382F492F5A2F82B79927AA27BB27F7
:100CA000282B392B4A2B5B2BCD0DD11DE11DF11DBE
:100CB0002C173D074E075F0758F580910C05909162
:100CC0000D05A0910E05B0910F0585B78F7885BFF2
:100CD00085B7806885BF889585B78F7785BF8091F8
:100CE0000C0590910D05A0910E05B0910F05BA2F3E
:100CF000A92F982F882722B7332744275527822BDF
:100D0000932BA42BB52B8C179D07AE07BF07A8F21A
:100D1000DF91CF911F910F91FF90EF90DF90089599
:100D20008091080590910905A0910A05B0910B05E5
:100D3000BC01CD0108958091100590911105A091FD
:100D40001205B0911305BC01CD010895893031F42D
:100D50008FB582608FBD8FB58E7F0AC08A3019F43F
:100D60008FB5826002C08FB58D7F8FBD8FB58160DA
:100D70008FBD1BBC1ABC19BC18BC08959C018FB553
:100D80008E7F8FBD8FB582608FBD8EB588608EBD22
:100D90008EB580618EBD37BD26BD1BBC1ABC19BC8B
:100DA00018BC08958FB58F778FBD8FB58F7B8FBDA2
:100DB00008958FB58F7D8FBD8FB58F7E8FBD0895C0
:100DC0008FB58D7F8FBD8FB58E7F8FBD0E94D20670
:100DD0000E94D90608958FB580688FBD8FB58F7B2F
:100DE0008FBD08958FB580628FBD8FB58F7E8FBD0B
:100DF00008959BBD8ABD089599BD88BD08951F9231
:100E00000F920FB60F9211242F933F934F935F933E
:100E10006F937F938F939F93AF93BF93EF93FF93C2
:100E20008091080590910905A0910A05B0910B05E4
:100E30000196A11DB11D8093080590930905A0930B
:100E40000A05B0930B0580910C0590910D05A091BA
:100E50000E05B0910F050196A11DB11D80930C05E3
:100E600090930D05A0930E05B0930F058091F801A6
:100E70009091F901892B29F0E091F801F091F901A5
:100E80000995FF91EF91BF91AF919F918F917F91C4
:100E90006F915F914F913F912F910F900FBE0F90E7
:100EA0001F9018951F920F920FB60F9211242F9337
:100EB0003F934F935F936F937F938F939F93AF93E2
:100EC000BF93EF93FF938091FA019091FB01892BDF
:100ED00029F0E091FA01F091FB010995FF91EF9162
:100EE000BF91AF919F918F917F916F915F914F9142
:100EF0003F912F910F900FBE0F901F9018951F924A
:100F00000F920FB60F9211242F933F934F935F933D
:100F10006F937F938F939F93AF93BF93EF93FF93C1
:100F20008091100590911105A0911205B0911305C3
:100F30000196A11DB11D8093100590931105A093FA
:100F40001205B09313058091020290910302892B40
:100F500029F0E0910202F09103020995FF91EF91CF
:100F6000BF91AF919F918F917F916F915F914F91C1
:100F70003F912F910F900FBE0F901F9018951F92C9
:100F80000F920FB60F9211242F933F934F935F93BD
:100F90006F937F938F939F93AF93BF93EF93FF9341
:100FA0008091060290910702892B29F0E0910602B8
:100FB000F09107020995FF91EF91BF91AF919F9139
:100FC0008F917F916F915F914F913F912F910F90F2
:100FD0000FBE0F901F9018951F920F920FB60F9291
:100FE00011242F933F934F935F936F937F938F932E
:100FF0009F93AF93BF93EF93FF938091FC019091E8
:10100000FD01892B29F0E091FC01F091FD0109958A
:10101000FF91EF91BF91AF919F918F917F916F91D0
:101020005F914F913F912F910F900FBE0F901F90A6
:1010300018951F920F920FB60F9211242F933F9382
:101040004F935F936F937F938F939F93AF93BF93D0
:10105000EF93FF938091FE019091FF01892B29F07E
:10106000E091FE01F091FF010995FF91EF91BF9191
:10107000AF919F918F917F916F915F914F913F9130
:101080002F910F900FBE0F901F9018951F920F92E7
:101090000FB60F9211242F933F934F935F936F934B
:1010A0007F938F939F93AF93BF93EF93FF93809121
:1010B000000290910102892B29F0E0910002F09149
:1010C00001020995FF91EF91BF91AF919F918F918F
:1010D0007F916F915F914F913F912F910F900FBE34
:1010E0000F901F9018951F920F920FB60F92112418
:1010F0002F933F934F935F936F937F938F939F9320
:10110000AF93BF93EF93FF938091040290910502F8
:10111000892B29F0E0910402F09105020995FF91D5
:10112000EF91BF91AF919F918F917F916F915F915F
:101130004F913F912F910F900FBE0F901F901895D8
:1011400096B1987F982B96B9089527B12F73992758
:1011500036E0880F991F3A95E1F7282B27B90895B3
:10116000379A359886E00E94A00881E00E94A50881
:101170003D98339A109214057894089533983798CF
:10118000089597B1907E8F71982B97B90895349AEE
:10119000369A089586B199278074907008951092B8
:1011A000140597B1907E8F71982B97B9349A369A1F
:1011B0003699FECF84B1282F332785B19927982FF0
:1011C0008827822B932B08950E94CF0896958795A8
:1011D00096958795992708951F920F920FB60F92B3
:1011E00011248F938FEF809314058F910F900FBE72
:1011F0000F901F90189581E890E00E949C0308953D
:1012000084E890E00E949C03089599279F938F9310
:1012100089E890E09F938F9381E08F930E94B004C0
:101220000F900F900F900F900F900895882319F052
:101230008FE890E002C086E990E09F938F9381E071
:101240008F930E94B0040F900F900F900895262F57
:1012500033273F932F9399279F938F938DE990E0A6
:101260009F938F9381E08F930E94B0048DB79EB7B8
:1012700007960FB6F8949EBF0FBE8DBF08951092CB
:1012800019051092150510921A0510921705109263
:1012900016051092180508950F931F939C018B015A
:1012A000909118058FE0989FC0011124B901885FC3
:1012B0009D4F0E94471480911805E82FFF27EE0FDD
:1012C000FF1FE05AFB4F118300838F5F8093180547
:1012D0001F910F9108959093B1048093B0040895E5
:1012E000CF93DF93C2ECD0E0FE018491882361F0BC
:1012F000FE0121968491E091B004F091B10409952A
:10130000FE0184918823A1F7DF91CF9108950F9377
:101310001F93CF93E091B004F091B1048DE0099553
:101320000E947009C09115050BE115E0C150CF3F37
:1013300051F0E091B004F091B104D8018D918D018C
:101340000995C150B0F7CF911F910F91089599273A
:10135000009719F0019761F0089580911B0588238B
:10136000D9F06BE175E08BE695E00E944714089593
:101370006BE675E08BE195E00E944714EBE1F5E048
:1013800001900020E9F73197EB51F540E093150506
:10139000E0931A050E9487090895CF93DF93C8EB65
:1013A000D0E0FE018491882349F0FE0121968491CA
:1013B000E091B004F091B1040995F3CFCBE1D5E011
:1013C00080911B0509C0803249F0E091B004F09192
:1013D000B1048991099588818823A9F7E091B00427
:1013E000F091B1048AE30995E091B004F091B10461
:1013F00080E20995C6EAD0E0FE018491882349F095
:10140000FE0121968491E091B004F091B104099518
:10141000F3CFE091B004F091B1048DE00995E09133
:10142000B004F091B1048AE00995DF91CF9108955D
:10143000FF920F931F93CF93DF9300E0802F0E94C2
:10144000A70980911B05803299F1882389F10F5FEC
:10145000E02FFF27E55EFA4FE081E03211F0EE2346
:10146000B1F7002371F424C0E12FFF27EE0FFF1F17
:10147000E05AFB4F80819181909317058093160568
:1014800019C010E0F09018051F1580F4C8E0D2E0F4
:10149000802F9927AC016BE175E0CE010E944E14BC
:1014A000892B11F31F5F2F961F1590F30E94CD0912
:1014B0000E947009DF91CF911F910F91FF900895C5
:1014C0001F93CF93182F20911905223009F045C0A2
:1014D00099278234910581F08334910524F4813475
:1014E000910541F037C08334910551F08434910562
:1014F00011F130C081E001C0822F0E94A7092AC0EB
:1015000090911A0580911505E091B004F091B10415
:101510009817F0F49F5F90931A058BE10995E0917D
:10152000B004F091B1048BE50995E091B004F0911D
:10153000B10483E40EC080911A05E091B004F091EB
:10154000B104882329F0815080931A0588E001C0F6
:1015500087E0099510921905EBC0213021F48B35F5
:1015600011F482E0E3C010921905812F80528F356B
:1015700008F04DC090911A05809115059817B1F4A7
:10158000E091B004F091B104812F099580911A0582
:10159000E82FFF27E55EFA4F10838F5F80931A05CF
:1015A000809115058F5F80931505C2C08F5F809372
:1015B0001505C82F981760F4A82FBB27A55EBA4F52
:1015C000FD01319780818C93C150DF019C17C0F3DE
:1015D00080911A05E82FFF27E55EFA4F10838F5F91
:1015E00080931A050E948709C0911A0580911505FC
:1015F000C81708F09DC0E091B004F091B10488E0F4
:101600000995CF5F80911505C817A8F391C01D30CB
:1016100011F5E091B004F091B104812F0995E091AA
:10162000B004F091B1048AE0099580911505E82F86
:10163000FF27E55EFA4F10828F5F8093150580913A
:101640001A058F5F80931A050E94180A10921505DB
:1016500010921A056DC0183009F063C080911A0508
:10166000882309F457C0909115058917E9F4E09192
:10167000B004F091B104812F0995E091B004F0918C
:10168000B10480E20995E091B004F091B104812F9A
:1016900009958091150581508093150580911A0553
:1016A000815080931A0544C0915090931505815044
:1016B00080931A05C82F891748F4E82FFF27E55EA5
:1016C000FA4F81818193CF5FC917D8F30E948709B0
:1016D000E091B004F091B10480E20995C0911A053F
:1016E0002C2F332780911505992701962817390744
:1016F000FCF4E091B004F091B10488E00995CF5F6B
:101700002C2F332780911505992701962817390723
:1017100084F30EC0E091B004F091B10487E0099524
:1017200007C01F3729F01B3119F481E08093190598
:10173000CF911F910895E0911605F091170530970C
:1017400039F0099510921705109216050E9470093C
:101750000895382F90E080911B05803239F49F5F07
:10176000E92FFF27E55EFA4F8081F7CF20E02317AE
:10177000B0F403C0E03241F09F5FE92FFF27E55E40
:10178000FA4FE081EE23B1F7E92FFF27E55EFA4F2C
:101790008081803211F49F5FF7CF2F5FE8CF892FD0
:1017A0009927855E9A4F0895CF93DF93CDB7DEB723
:1017B00022970FB6F894DEBF0FBECDBF0E94A90BD3
:1017C0004AE050E0BE016F5F7F4F0E944213DC0190
:1017D000CB01BC01CD0122960FB6F894DEBF0FBE3F
:1017E000CDBFDF91CF910895CF93DF93CDB7DEB713
:1017F00022970FB6F894DEBF0FBECDBF0E94A90B93
:1018000040E150E0BE016F5F7F4F0E944213DC0158
:10181000CB01BC01CD0122960FB6F894DEBF0FBEFE
:10182000CDBFDF91CF910895E199FECF9FBB8EBBD5
:101830006DBBE29AE19A0895EF92FF921F93CF93C6
:10184000DF93CDB7DEB721970FB6F894DEBF0FBE9A
:10185000CDBFEE24FF240E94000960E081E00E94D9
:1018600027098DEE91E00E949C030E943F098CE6BF
:1018700092E00E946B0966EF7CE086E890E00E94AF
:101880004C0967EF7CE08BE890E00E944C096BEF1D
:101890007CE080E990E00E944C0968E37DE085E906
:1018A00090E00E944C096AE47DE088E990E00E94A3
:1018B0004C0965E97DE08BE990E00E944C096FEAF4
:1018C0007DE08EE990E00E944C0968E57EE081EAC7
:1018D00090E00E944C096FEF7CE085EA90E00E9466
:1018E0004C0969EE7DE088EA90E00E944C0963EFC4
:1018F0007DE08CEA90E00E944C0962E07EE080EBA3
:1019000090E00E944C096CE07EE084EB90E00E9445
:101910004C0966E17EE087EB90E00E944C0965E2AD
:101920007EE08AEB90E00E944C0964E37EE08DEB60
:1019300090E00E944C0965E37EE080EC90E00E941C
:101940004C098DE00E94600A8FEF80930B0603C064
:1019500089810E94600ACE0101960E947502182FAB
:101960008823B1F70894E11CF11C89EEE81683E0A6
:10197000F80610F0EE24FF248091B2048823A1F031
:1019800060917B0080E090E00E94140C6091BC04A8
:1019900081E090E00E94140C6091BB0482E090E032
:1019A0000E94140C1093B2040E949B0B80910B06B2
:1019B000882389F60E94B0038DEF91E09F938F9367
:1019C00081E08F930E94B0040F900F900F902196AA
:1019D0000FB6F894DEBF0FBECDBFDF91CF911F9140
:1019E000FF90EF90089510920B060895089580E0FF
:1019F0000E94A508089581E00E94A5080895FF921D
:101A00000F931F9329B386B3F3B200B399279F9323
:101A10008F93822F99279F938F938FE092E09F93CC
:101A20008F9311E01F930E94B0048DB79EB7079665
:101A30000FB6F8949EBF0FBE8DBF802F99279F933E
:101A40008F938F2D99279F938F9388E192E09F9397
:101A50008F931F930E94B0048DB79EB707960FB661
:101A6000F8949EBF0FBE8DBF1F910F91FF900895F8
:101A700089B399279F938F9383E292E09F938F93EB
:101A800081E08F930E94B0040F900F900F900F9001
:101A90000F9008951F93CF93DF9386B399279F9359
:101AA0008F9382E392E09F938F9381E08F930E94C4
:101AB000B0040F900F900F900F900F90C1E5D6E0FB
:101AC000899199279F938F9383E492E09F938F93BB
:101AD00011E01F930E94B0040F900F900F900F9091
:101AE0000F9086E0CA35D80759F354F3809162000D
:101AF00099279F938F9387E492E09F938F931F93EF
:101B00000E94B0040F900F900F900F900F9086E5F9
:101B100092E09F938F931F930E94B0040F900F90B9
:101B20000F90DF91CF911F9108951F9383B3992751
:101B30009F938F9389E592E09F938F9311E01F937A
:101B40000E94B004812F0E94D40BDC01CB0185BB25
:101B50000F900F900F900F900F901F9108951F936B
:101B60000E94B00380B399279F938F938EE592E0F4
:101B70009F938F9311E01F930E94B004812F0E94C6
:101B8000D40BDC01CB0182BB0F900F900F900F9014
:101B90000F901F91089581E00E94D40BDC01CB01CE
:101BA0008CBF08950895089581E00E94D40BDC0154
:101BB000CB019C01832F99278BBD2ABD089581E01D
:101BC0000E94D40BDC01CB0190937D0080937C00BC
:101BD000089581E00E94D40BDC01CB019093780042
:101BE00080937700089581E00E94D40BDC01CB0143
:101BF0008093760082E00E94D40BDC01CB018093BD
:101C00007500089581E00E94D40BDC01CB01909314
:101C10007A0080937900089581E00E94D40BDC0162
:101C2000CB019093740080937300089581E00E942B
:101C3000D40BDC01CB018093610082E00E94D40BC5
:101C4000DC01CB0180936000089581E00E94D40BF9
:101C5000DC01CB018093720182E00E94D40BDC0195
:101C6000CB0180937101089508958FE790E080542F
:101C7000904097FFFCCF83E692E09F938F9381E0A3
:101C80008F930E94B0040F900F900F908FE790E019
:101C90008054904097FFFCCF86E692E09F938F930D
:101CA00081E08F930E94B0040F900F900F900895E1
:101CB000FF920F931F93CF93DF9320E030E0CFED9F
:101CC000D4E0899199919F938F9389010F5F1F4F62
:101CD0001F930F9389E692E09F938F9391E0F92EE3
:101CE000FF920E94B0048DB79EB707960FB6F89486
:101CF0009EBF0FBE8DBF98010830110510F385E718
:101D000092E09F938F93FF920E94B0040F900F90E8
:101D10000F90DF91CF911F910F91FF90089508953B
:101D2000282F3327E091BF04F091C0042E1B3F0BF6
:101D30008091600099276091C1047091C204689FEE
:101D4000A001699F500D789F500D1124CA01B6E083
:101D500095958795BA95E1F7281B390B3093C40404
:101D60002093C30480916100482F5527429FC001F2
:101D7000439F900D529F900D1124A6E09595879555
:101D8000AA95E1F7860F971F9093C2048093C10430
:101D9000489F9001499F300D589F300D1124C90173
:101DA00036E0959587953A95E1F78E0F9F1F9093B2
:101DB000C0048093BF0424E0959587952A95E1F7A8
:101DC000805899270895CF93DF93CDB7DEB7229738
:101DD0000FB6F894DEBF0FBECDBF8091C6048F5FF3
:101DE0008093C604843040F01092C604CE01019660
:101DF0000E941C128093C50422960FB6F894DEBF91
:101E00000FBECDBFDF91CF910895EF92FF920F9358
:101E10001F93CF93DF93CDB7DEB766970FB6F894D5
:101E2000DEBF0FBECDBF8B0160E070E0FE013196DA
:101E3000AF0123ECE22E20E0F22E26E1D7010D9037
:101E40007D01DA010D92AD012150C1F7880F991F74
:101E5000E80FF91F20813181200F311F8091790017
:101E600090917A00280F391F33232CF46150704071
:101E7000245F3F4FF9CF2C3031052CF06F5F7F4F3F
:101E80002C503040F8CFC901820F931FFC01EB5357
:101E9000FF4F24913327322F22278A539F4FFC0173
:101EA0008491280F311D309364002093630040E03B
:101EB00050E084E090E0861B970B481759075CF4CC
:101EC000369527954F5F5F4F48175907CCF33093EE
:101ED0006400209363008091630090916400669693
:101EE0000FB6F894DEBF0FBECDBFDF91CF911F912B
:101EF0000F91FF90EF9008951F93CF93DF93C0E071
:101F0000D0E08091C7049927009719F00197E1F07C
:101F100031C023B390E131E0E1E5F6E0822F89237F
:101F200011F0108201C030839695319646E0E53578
:101F3000F407A1F39CF381E08093C704AC98AD9AB9
:101F400019C02093620025C023B390E131E0E6E59B
:101F5000F6E0822F892311F0108201C0308396951C
:101F6000319656E0EA35F507A1F39CF31092C704C9
:101F7000AC9AAD9883E68093620020E030E0E1E522
:101F8000F6E081918823E9F62F5F3F4F2A30310533
:101F9000C4F390916200933629F41092C804109211
:101FA000BD0436C09F5F9093C80491509A30A0F44E
:101FB000E92FFF27EF5AF94F8181882369F0993083
:101FC00030F48281882319F0C2E0D0E002C0C1E081
:101FD000D0E01092BD0420C0993060F4E92FFF27B3
:101FE000EF5AF94F8281882329F081E08093BD0464
:101FF00010E012C0993060F4E92FFF27EF5AF94F33
:102000008381882329F081E08093BD04182F04C0C8
:102010001092BD04C0E0D0E02091C8048091D900A6
:10202000281769F49091BD048091DA00981739F46B
:102030008091C9049927C817D90709F492C08091E3
:10204000BD049927009719F0019759F080C0BE018F
:10205000822F99270E94050F90936400809363005C
:1020600076C0CE014896BC01822F99270E94050FA9
:102070009C01909364008093630090932B0680935F
:102080002A06880F991F90932D0680932C06A9018C
:10209000480F591F50932F0640932E06812F9927E2
:1020A0008130910531F1823091051CF4892B21F0AA
:1020B0004EC00297D9F14BC08BE490E0289FA0015D
:1020C000299F500D389F500D11249A01E6E0369556
:1020D0002795EA95E1F73093310620933006C90140
:1020E000880F991F9093330680933206820F931FB7
:1020F0002AC0C901880F991F880F991F820F931F4B
:10210000969587959695879590933106809330069E
:102110009C01220F331F3093330620933206280F81
:10212000391F309335062093340611C0CA019695A5
:1021300087959093310680933006509333064093F1
:102140003206840F951F9093350680933406809154
:10215000C8048093D9008091BD048093DA00C093B5
:10216000C9048091C8049927DF91CF911F910895E8
:10217000CF93DF938091CA048F5F83708093CA04EA
:10218000882311F40E94E30E0E947C0F8091BD040D
:1021900099278130910509F44FC0823091051CF4D4
:1021A000892B29F07EC0029709F443C07AC0809140
:1021B000B4049091B5042091630030916400820FC3
:1021C000931F9093B5048093B4042091B904309187
:1021D000BA042817390728F48091750083BD959AB1
:1021E00004C08091760083BD95988091B60490914B
:1021F000B70401969093B7048093B60420916500CC
:10220000309166002817390708F04BC01092B704C8
:102210001092B6048091770090917800825A9E4F78
:1022200090937800809377009093BA048093B904D8
:1022300038C00E94931234C040E050E0CAE2D6E0B9
:10224000ACE3B6E08D919C91119729913991820F61
:10225000931F8D939D93E92FFF27EE7FF070E3513D
:10226000FF4F8491480F511D86E0A634B80751F303
:102270004CF34050534082E04030580714F04FEF89
:1022800051E08EEF4130580714F441E05EEF4150C9
:102290005E4F5595479555954795842F0E94900E12
:1022A00083BDDF91CF91089589B78D7F89BF68EB9A
:1022B00070E187E00E94E8059AE093BF8DE28CBF51
:1022C00089B7826089BF89B78F7E89BF89B78F77C9
:1022D00089BF89E785BD93BD0895CFE5D8E0DEBF0E
:1022E000CDBF0E94480260E071EE80E090E00E9465
:1022F00018028CE692E00E9444030E94B0080E94FB
:10230000FB0888E792E09F938F9381E08F930E9470
:10231000B0041ABA1BBA17BA9FEF98BB80E684BB09
:102320008FE185BB91BB12BA969A0E9418130E9446
:1023300054110E941C0C0F900F900F9080E090E0C1
:102340000C940E150895089508950895E199FECF0F
:102350009FBB8EBBE09A8DB399270895BF92CF9211
:10236000DF92EF92FF920F931F93CF93DF93EE24B0
:10237000FF24670100E010E0E601CE010E94A611F3
:1023800099279F938F9383E992E09F938F9331E0F6
:10239000B32EBF920E94B0040F900F900F900F9039
:1023A0000F900F5F1F4F21960032110534F387E91C
:1023B00092E09F938F93BF920E94B0040F900F9072
:1023C0000F900894E11CF11C80E290E0C80ED91E29
:1023D0001E141F047CF6DF91CF911F910F91FF9087
:1023E000EF90DF90CF90BF9008954091DB00509127
:1023F000DC00BA016627770F661F7727CA01807055
:10240000907484E0989F812D992711249A0120705F
:102410003071232F332722952F7086279727822705
:1024200093279A01220F331F282B392B3093DC007E
:102430002093DB00C9010895FC0184B1682F772740
:1024400085B1482F55279A01237030708091EF0491
:102450009927009719F00197A1F160C08091F004CD
:102460008F5F8093F004909170018917E0F4322F10
:102470002227330F330F660F771F660F771F260F44
:10248000371F3093CE042093CD0441FF03C080E07A
:1024900098E002C080E098EF282739273093CE04D7
:1024A0002093CD043BC01092F0048091F1048F5F23
:1024B00087708093F104805C87B981E08093EF049A
:1024C0002DC01092EF04522F4427460F571F5183FF
:1024D000408384E487B98091F104682F7727CB018A
:1024E000860F971FFC01E152FB4F51834083FC0193
:1024F000E153FB4F808191819A01281B390B37FFF3
:1025000003C0309521953F4F80916F01992728177F
:10251000390714F051834083CB01089586EC86B9C6
:1025200083E690E00895EF92FF920F931F93CF936D
:10253000DF938091F8069091F906FC0136E0F6955C
:10254000E7953A95E1F7EE0FFF1FE650F94FC0818E
:10255000D1812091F6063091F706280F391F30936C
:10256000F9062093F80640E12030340728F03F7048
:102570003093F9062093F806C058DF4F8091F3049A
:102580008F5F8093F304843008F449C01092F30401
:1025900080917201082F11276091F204A62FBB27AA
:1025A000FD01FF96EF73F070EE0FFF1FE650F94F3D
:1025B00080819181089F9001099F300D189F300DF7
:1025C000112480917101482F5527FD01EA0FFB1F4F
:1025D000E650F94F80819181489F7001499FF00C2E
:1025E000589FF00C11242E0D3F1D1196AF73B07043
:1025F000AA0FBB1FA650B94F8D919C91089FA001B7
:10260000099F500D189F500D1124240F351F232FA3
:102610003327318320836F5F6F736093F2048C2FB5
:102620009927DF91CF911F910F91FF90EF9008951F
:102630001092F9061092F806E6E7F6E0AAEFB6E087
:102640001D921D921192119286E0E43FF807C1F3AA
:10265000BCF389E190E09093F7068093F6068CE056
:1026600090E09093F9068093F8068FE090E09093C5
:10267000FB068093FA0688E090E09093FD06809335
:10268000FC060895A0E0B0E0E8E4F3E10C94D9146E
:102690008C012B01EA01EE246115710519F0FB0193
:1026A00091838083209749F0CE010297839728F089
:1026B00060E070E080E090E0E5C0F801F1908F010B
:1026C0008F2D99270E94CC14892BB9F7FDE2FF16B4
:1026D00019F441E0E42E03C0FBE2FF1619F4F801FF
:1026E000F1908F01209719F0C031D10591F4F0E3FA
:1026F000FF1679F4F8018081883711F0883549F4A4
:10270000F801F1800E5F1F4FC0E1D0E0F2E0EF2A48
:102710000AC0209741F480E3F81619F4C8E0D0E02D
:1027200002C0CAE0D0E0C830D105E9F0C930D10517
:1027300024F4C230D105E9F022C0CA30D10521F01D
:10274000C031D10551F01BC03CECA32E3CECB32EA4
:102750003CECC32E3CE0D32E1FC0A12CB12CC12CCD
:1027600028E0D22E19C0A12CB12CC12C90E1D92E79
:1027700013C0A12CB12CC12C80E4D82E0DC09E0119
:10278000442737FD4095542F60E070E080E090E8EA
:102790000E948F1459016A0120E030E040E050E0CF
:1027A00060E03E01882477FC8094982C8F2D805324
:1027B0008A3010F4F82E0DC08F2D81548A3118F410
:1027C000E9ECFE0E06C08F2D81568A3148F5F9EAF4
:1027D000FF0E8F2D99278C179D0714F567FD1CC0E0
:1027E000A216B306C406D506A0F0CA01B901A40119
:1027F00093010E945C149B01AC012F0D311D411D02
:10280000511D213080E0380780E0480780E85807F4
:1028100010F06FEF01C061E0F801F1908F01C6CFB9
:102820004114510461F0662319F00150104004C0B6
:10283000E1FE05C002501040F201118300838E2D8D
:10284000992767FF07C080FF11C020E030E040E01B
:1028500050E810C080FF08C05095409530952195F4
:102860003F4F4F4F5F4F0CC057FF0AC02FEF3FEF56
:102870004FEF5FE782E290E090937B0780937A07C7
:10288000CA01B901E0E1CDB7DEB70C94F514FB0144
:10289000DC0101900D920020E1F70895FB01DC01BD
:1028A0004150504030F08D910190801919F4002072
:1028B000B9F7881B990B0895629FD001739FF001AF
:1028C000829FE00DF11D649FE00DF11D929FF00DC0
:1028D000839FF00D749FF00D659FF00D9927729FF7
:1028E000B00DE11DF91F639FB00DE11DF91FBD0182
:1028F000CF0111240895AA1BBB1B51E107C0AA1FD9
:10290000BB1FA617B70710F0A61BB70B881F991F90
:102910005A95A9F780959095BC01CD010895A1E243
:102920001A2EAA1BBB1BFD010DC0AA1FBB1FEE1F49
:10293000FF1FA217B307E407F50720F0A21BB30B94
:10294000E40BF50B661F771F881F991F1A9469F710
:1029500060957095809590959B01AC01BD01CF016C
:10296000089597FB092E05260ED057FD04D0D7DF1A
:102970000AD0001C38F450954095309521953F4F72
:102980004F4F5F4F0895F6F790958095709561953C
:102990007F4F8F4F9F4F0895911106C0803219F0DD
:1029A00089508550D0F708959927882708952F9248
:1029B0003F924F925F926F927F928F929F92AF92CF
:1029C000BF92CF92DF92EF92FF920F931F93CF931C
:1029D000DF93CDB7DEB7CA1BDB0B0FB6F894DEBFB3
:1029E0000FBECDBF09942A88398848885F846E84D9
:1029F0007D848C849B84AA84B984C884DF80EE8023
:102A0000FD800C811B81AA81B981CE0FD11D0FB62B
:0E2A1000F894DEBF0FBECDBFED010895FFCFDD
:102A1E000A3C63D007BC02F00AC012901AA82FC05D
:102A2E005D606D2E00FF0A0080D0FFFFE8030A00F4
:102A3E00FF000000FF0068656C7000617265660043
:102A4E006176636300706100706200706300706491
:102A5E00006164630070700070776D00706C6800C8
:102A6E006F666600616D00737600616200736200CE
:102A7E006473000A000C000F0011001300160018FA
:102A8E00001B001D001F00220063630100010057A0
:102A9E00012F01210113010901FF003D014B010C22
:102AAE0000070007000700050005000600000000F3
:102ABE0000040005000700090000000300050007E0
:102ACE00000A000000020003000500070008000BCA
:102ADE00000000020003000500070008000A0000C5
:102AEE0000020004000500070009000B00000002B0
:102AFE0000030005000600080009000000020004A3
:102B0E0000060008000A0000000100020003000495
:102B1E0000050006000700080009000A000B00145B
:042B2E000A32040063
:00000001FF
